:107800000C943B3C0C94793C0C94793C0C94793C62
:107810000C94793C0C94793C0C94793C0C94793C14
:107820000C94793C0C94793C0C94793C0C94793C04
:107830000C94793C0C94793C0C94793C0C94793CF4
:107840000C94793C0C94793C0C94793C0C94793CE4
:107850000C94793C0C94793C0C94793C0C94793CD4
:107860000C94793C0C94793C437934436F6465A063
:10787000000121B0012011241FBECFEFD8E0DEBFF0
:10788000CDBF84B714BE20914F02309150024FE01B
:1078900098E10FB6F894A895909360000FBE4093BE
:1078A000600080FD07C081FD0DC083FF03C0283745
:1078B000324D41F0E0E0F0E085919491019611F0B5
:1078C0000C94000011E0A0E0B1E0E0EEFFE702C0A0
:1078D00005900D92A230B107D9F722E0A2E0B1E005
:1078E00001C01D92AF34B207E1F70E94003E0C9434
:1078F000EE3F0C94A63C87E084B915B88FEC87B9AD
:1079000018B88CE98AB91BB8579A5F9A85E08093BA
:1079100081001092C00088E18093C10083E290E072
:107920009093C5008093C400089588E792ED9093EA
:10793000500280934F0298E088E10FB6F894A89522
:10794000809360000FBE90936000FFCFF8940E9478
:10795000953C1092500210924F0298E088E10FB6C9
:10796000F894A895809360000FBE90936000FFCFBD
:107970009091C00095FFFCCF8093C60008950F93AF
:107980001F93CF93DF9300D0CDB7DEB78C01A62F26
:10799000B0E020E030EC48EA50E00E94A23F20E452
:1079A0003FE140E050E00E94803F3A832983898193
:1079B0009A81892B21F481E090E09A8389838981DF
:1079C0009A8120E8A0ECB0E00C90022211F401971B
:1079D000D9F79A83898389819A81892B31F08091A3
:1079E000C600F801808381E001C080E00F900F9015
:1079F000DF91CF911F910F910895882319F0AFE483
:107A0000B1E002C0AFECB1E020E8829FC0011124D8
:107A10009D0120583F4F8A1B9B0BFC01EA0FFB1F67
:107A2000E491ED93A217B307C1F708950F931F9345
:107A3000CF93DF93882319F0AFE4B1E002C0AFEC3D
:107A4000B1E020E8829FC001112423E0FC012093D3
:107A50005700E89507B600FCFDCFAD0140585F4FD9
:107A6000ED0161E08C010A1B1B0BF801EC0FFD1FFF
:107A7000298130E0322F22277881270F311D09011B
:107A800060935700E895112422964C175D0769F71B
:107A900025E0FC0120935700E89507B600FCFDCFD8
:107AA00021E120935700E89520E030E04D91FC0162
:107AB000E20FF31FE4914E1307C02F5F3F4F2038B2
:107AC0003105A1F781E001C080E0DF91CF911F91E6
:107AD0000F910895DF92EF92FF920F931F93CF9330
:107AE000DF9300D0CDB7DEB79091030183E0892703
:107AF00080930301909106019093040190910701F6
:107B000090930501909100019093060190910101DD
:107B10009093070180FF04C010910B01165F01C014
:107B20001AE0E2E0F1E08FEF90E0191779F021918F
:107B3000822728E0382F369580FD02C080E001C002
:107B40008CE883272150B1F79F5FEFCFE12FF0E062
:107B5000EE5FFE4F8083E0908400F090850084E724
:107B6000E81A85EFF80A00E063E0CE0102960E9471
:107B7000BF3C811116C000E0E02FF0E0EE5FFE4F49
:107B8000D0808D2D0E94B83C61E0CE0101960E940C
:107B9000BF3C882331F08981D81203C00F5F1017D2
:107BA00058F7101748F080918400909185008E1945
:107BB0009F0918161906C4F60F900F90DF91CF9108
:107BC0001F910F91FF90EF90DF900895E2E0F1E0B8
:107BD0006681862F90E0A0E0B0E0DC01992788273D
:107BE0002085820F911DA11DB11D278130E0322F0C
:107BF0002227BC01CD01620F731F811D911D0895C5
:107C0000CF93DF93CDB7DEB729970FB6F894DEBFD9
:107C10000FBECDBF0E947B3C44E050E062E070E0CC
:107C2000CE0105960E94BC3F8F81809528852095C6
:107C30009D81891303C09E81291789F08FEF898365
:107C400088E78A831B8287E88C8344E050E062E007
:107C500070E0CE0101960E94CC3F98E78FEF8093B1
:107C600000019093010100E010E0C0908400D090EA
:107C7000850020E7C21A21E8D20A43E1F42E8F2DB5
:107C80008271823119F48BB180588BB9F394A89525
:107C900080918400909185008C199D091816190611
:107CA00014F410924E0169E1CE0101960E94BF3C8E
:107CB000882329F35F9AA89589818A3AF1F6FF24EF
:107CC000FA943AE4E32EB12C8981EB2DF0E0EE5FDB
:107CD000FE4F808391E0B91206C0982F9695969535
:107CE000903381F026C0E9E0BE120CC0813408F563
:107CF0009091030190FF02C0982F01C090E02AE00C
:107D0000E22EE90EF82688E02F2D2695F0FC02C021
:107D100090E001C09CE8F22EF9268150A9F763E0BB
:107D2000CE0101960E94BF3C882319F0B394BE1483
:107D300058F2BE10A2CF89818F119FCFF09003011E
:107D4000F1FE9BCF9091000180910401981395CF93
:107D5000909101018091050198138FCF0E94E63D1B
:107D6000603FFFEF7F078F07910570F030910B01A7
:107D7000E62E2FE32F0D223070F4605FACE0B1E00F
:107D800080E0673008F44DC080910301815C82304F
:107D900008F055C06ACF313011F56D7F683F09F0AA
:107DA0004EC080910C018E3509F049C028EFE212D7
:107DB0000BC080914E01882339F080914D010E94C3
:107DC000163D80E00E94163D0E946A3D8AEFE8124F
:107DD00003C00E94953CD8CF0E94A93CD5CF323039
:107DE00071F59CEFE9122BC0E0900C01EE2039F107
:107DF000F0900D01FF2019F10E946A3DE092000110
:107E0000F0920101E982FA82E094EB82F094FC8224
:107E100044E050E062E070E0CE0101960E94CC3F69
:107E2000B3CFE62FF0E0E159F748E491ED936F5FAF
:107E30008F5F831708F4A5CF0E946A3DA5CF0E94EB
:107E4000E63D4B015C01611578478105910508F01D
:107E50000CCF80914E01811111C0E1E0E0934E0101
:107E600010924D010E94FD3C07B600FCFDCFF99930
:107E7000FECF83E0F80180935700E8957501640117
:107E8000C9863C2C381880910B013816B0F52601B4
:107E9000370187E076946794579447948A95D1F791
:107EA000242C80914D01481679F0811106C02220C2
:107EB00049F0842D0E94FD3C05C00E94163D8111B1
:107EC000F6CFD3CE40924D0189858F7720914D0119
:107ED00090E0E32DF0E0DC01211103C0A153BE4F7F
:107EE00002C0A15BBE4FE45FFE4F20812C93FFEFE9
:107EF000CF1ADF0AEF0AFF0AC3CF0E946A3DB5CE50
:107F0000A1E21A2EAA1BBB1BFD010DC0AA1FBB1F9D
:107F1000EE1FFF1FA217B307E407F50720F0A21B0F
:107F2000B30BE40BF50B661F771F881F991F1A947C
:107F300069F760957095809590959B01AC01BD01A6
:107F4000CF0108950E94AD3FA59F900DB49F900D65
:107F5000A49F800D911D11240895A29FB001B39F8D
:107F6000C001A39F700D811D1124911DB29F700D42
:107F7000811D1124911D0895DC01CB01FC01F999AB
:107F8000FECF06C0F2BDE1BDF89A319600B40D9265
:107F900041505040B8F70895DC01A40FB51F41507F
:107FA000504048F0CB01840F951F2E910E94DD3F79
:107FB00041505040D0F70895262FF999FECF92BD39
:107FC00081BDF89A019700B4021639F01FBA20BD9E
:107FD0000FB6F894FA9AF99A0FBE0895F894FFCF65
:027FE000FFFFA1
:040000030000780081
:00000001FF
